:020000040000FA
:040000006B303A28FF
:08000800A000030EA100831209
:1000100005191028831601178312B23081002B288E
:1000200083160113831203140B190310A80DA90DD5
:10003000AA0DAB0DAC0DAC16FF302C02031D2B2806
:10004000FA302B02031D2B2831152A08AF0029088E
:10005000AE002808AD008B100B11210E8300A00EFE
:04006000200E090065
:0C007400203084008001840A6030040207
:10008000031C3C281230B000982183160C308505E3
:1000900087018312850187010730990000309A009B
:1000A000103083168E008312603083168F00831207
:1000B0000030831691008312C830831681008312AA
:1000C00031309000003083168C00831210308B008A
:1000D000831600309B001C141A088312BC00831680
:1000E00010309B001C141A088312BD00DC21810112
:1000F0008E018F010B118B100B108C018B178E2032
:1001000031199120B30B8C28031085190314B90DF4
:10011000F030390203191D21F5217F2864003210C7
:10012000080031110130B7008B13203037078316D8
:100130009B001C141A088312A40010303707831682
:100140009B001C141A088312A300A6000230A60606
:100150000030370783169B001C141A088312A20074
:10016000A7000130A7068B17321CBC2822090339CF
:10017000A200A309A409A50924082F02031D172919
:1001800023082E02031DEB2822082D02031D172928
:1001900001303702031DCF283D143E14A521023043
:1001A0003702031DD628BD143E14A921033037029F
:1001B000031DDD283D153E14AD2104303702031D1B
:1001C000E428BD153E14B12105303702031DEB288C
:1001D0003D163E14B52126082E02031D17292708B7
:1001E0002D02031D172901303702031DFA283D1087
:1001F0003E14B92102303702031D0129BD103E14FF
:10020000BD2103303702031D08293D113E14C121D1
:1002100004303702031D0F29BD113E14C5210530DE
:100220003702031D16293D123E14C9211729B70AAA
:10023000063037020318080094280130B600B300D6
:10024000B400B500B70085018701B1138E20B30B50
:100250004929031085190314B90DF0303902031927
:100260007029B40B4929013037020319CD2102301E
:1002700037020319D021033037020319D321043088
:1002800037020319D621053037020319D9219630D8
:10029000B400311D26293111321C53292D0903398F
:1002A000AD00AE09AF092F1C26298E018F010C1C51
:1002B00026290C102E1E26298B1320303707BB0051
:1002C0002F08BA00832110303707BB002E08BA0070
:1002D000832100303707BB002D08BA0083218B171C
:1002E00085018701B70AB60106303702031C2629AB
:1002F000DC2108003E1C08003E101030BB003D0809
:10030000BA00832108008B133A0883161C159A0043
:1003100083123B0883169B0055309D00AA309D0038
:100320009C1464009C1891291C1183128B170800DF
:10033000FF30D000D415D515D615D715D815D91539
:10034000DA15DB15DC15DD150800D2104E14CE10C1
:100350000800D2114E15CE110800D2124E16CE1240
:100360000800D2134E17CE130800D3104F14CF102D
:1003700008005210CE144E1008005211CE154E1126
:1003800008005212CE164E1208005213CE174E130A
:1003900008005310CF144F100800303085060800B5
:1003A00003308506080006308706080021308706DE
:1003B00008001830870608003D184E143D1CCE1466
:1003C000BD184E15BD1CCE153D194E163D1DCE1641
:1003D000BD194E17BD1DCE173D1A4F143D1ECF142B
:1003E0004E08D200CF00D30008008F080319080080
:1003F0008F01D00F372BD00A521C0D2A541D032A0F
:10040000D40154161B2AD41D082AD40154161B2AC1
:10041000541E1B2AD401D4141B2AD41C122AD40122
:1004200054151B2A541D172AD401D4151B2A541EF7
:100430001B2AD4015415D21C2C2A551D222AD50161
:1004400055163A2AD51D272AD50155163A2A551E82
:100450003A2AD501D5143A2AD51C312AD501551589
:100460003A2A551D362AD501D5153A2A551E3A2A5B
:10047000D5015515521D4B2A561D412AD601561637
:10048000592AD61D462AD6015616592A561E592AC9
:10049000D601D614592AD61C502AD6015615592AE7
:1004A000561D552AD601D615592A561E592AD60147
:1004B0005615D21D6A2A571D602AD7015716782A69
:1004C000D71D652AD7015716782A571E782AD701D3
:1004D000D714782AD71C6F2AD7015715782A571DA9
:1004E000742AD701D715782A571E782AD7015715AD
:1004F000521E892A581D7F2AD8015816972AD81DBE
:10050000842AD8015816972A581E972AD801D81439
:10051000972AD81C8E2AD8015815972A581D932A35
:10052000D801D815972A581E972AD8015815D21ED7
:10053000A82A591D9E2AD9015916B62AD91DA32ABF
:10054000D9015916B62A591EB62AD901D914B62A84
:10055000D91CAD2AD9015915B62A591DB22AD9017B
:10056000D915B62A591EB62AD9015915521FC72ABC
:100570005A1DBD2ADA015A16D52ADA1DC22ADA0115
:100580005A16D52A5A1ED52ADA01DA14D52ADA1CC7
:10059000CC2ADA015A15D52A5A1DD12ADA01DA15E0
:1005A000D52A5A1ED52ADA015A15D21FE62A5B1D12
:1005B000DC2ADB015B16F42ADB1DE12ADB015B167A
:1005C000F42A5B1EF42ADB01DB14F42ADB1CEB2A81
:1005D000DB015B15F42A5B1DF02ADB01DB15F42A35
:1005E0005B1EF42ADB015B15531C052B5C1DFB2AEB
:1005F000DC015C16132BDC1D002BDC015C16132BBD
:100600005C1E132BDC01DC14132BDC1C0A2BDC011D
:100610005C15132B5C1D0F2BDC01DC15132B5C1EF2
:10062000132BDC015C15D31C242B5D1D1A2BDD0163
:100630005D16322BDD1D1F2BDD015D16322B5D1E7D
:10064000322BDD01DD14322BDD1C292BDD015D1584
:10065000322B5D1D2E2BDD01DD15322B5D1E322B65
:10066000DD015D157A214E08D2004F08D3005008F5
:10067000D1000C305405031D05120C305505031D27
:1006800085120C305605031D05100C305705031D4F
:1006900085100C305805031D87100C305905031DBB
:1006A00007110C305A05031D07100C305B05031DA4
:1006B00087120C305C05031D07120C305D05031D0D
:1006C000871151080E020318912B12305405031D97
:1006D000051612305505031D851612305605031DEB
:1006E000051412305705031D851412305805031DDB
:1006F000871412305905031D071512305A05031DC2
:10070000071412305B05031D871612305C05031DAC
:10071000071612305D05031D8715FF3050020319BF
:1007200008008F08031D08008E2051080E02031CCC
:10073000912B18305405031D051206305405031D76
:10074000051618305505031D851206305505031D85
:10075000851618305605031D051006305605031D75
:10076000051418305705031D851006305705031D65
:10077000851418305805031D871006305805031DD1
:10078000871418305905031D071106305905031D3C
:10079000071518305A05031D071006305A05031DAA
:1007A000071418305B05031D871206305B05031D17
:1007B000871618305C05031D071206305C05031D03
:1007C000071618305D05031D871106305D05031DF2
:0407D0008715080081
:084000000200030002000600AB
:02400E00CC33B1
:10420000010078007A007C007E007B0079007F004E
:104210007D007A0078007E007C00FF00FF00FF0038
:104220000000F200F600FA00FE00F200F600FA00CC
:10423000FE00F200F600FA00FE00FF00FF00FF00A3
:10424000010005000500050005000900090009003E
:1042500009000D000D000D000D00FF00FF00FF0024
:10426000FF00FF00FF00FF00FF00FF00FF00FF0056
:10427000FF00FF00FF00FF00FF00FF00FF00FF0046
:10428000FF00FF00FF00FF00FF00FF00FF00FF0036
:10429000FF00FF00FF00FF00FF00FF00FF00FF0026
:1042A000FF00FF00FF00FF00FF00FF00FF00FF0016
:1042B000FF00FF00FF00FF00FF00FF00FF00FF0006
:1042C000FF00FF00FF00FF00FF00FF00FF00FF00F6
:1042D000FF00FF00FF00FF00FF00FF00FF00FF00E6
:1042E000FF00FF00FF00FF00FF00FF00FF00FF00D6
:1042F000FF00FF00FF00FF00FF00FF00FF00DD00E8
:00000001FF
